:020000040000FA
:1000000083018B018A019A28A000030EA1008301BD
:10001000051D1C282A08820725282E283628362860
:10002000362836283628362836283C2843284B28B8
:10003000532862286F287C28B33081000B110B10E5
:10004000210E8300A00E200E09004A1CA90A0B19DC
:10005000A901F63029070318AA0A1F280B19AA0AB2
:10006000AB01A901A601A701A8011F2803140B19C0
:100070000310A20DAA0A1F2803140B190310A20DC6
:100080002B0AAA071F2800300B190230AA002208E9
:10009000A300AB0A1F2800300B190230AA00220867
:1000A000A400AB0A1F280B1D5C280230AA002208FE
:1000B000A500AB0ACA151F28AA012208A5004A14E8
:1000C000CA111F280B1D6A280230AA002208A600A8
:1000D000AB0A1F28AA012208A6004A141F280B1DDC
:1000E00077280230AA002208A700AB0A1F28AA011D
:1000F0002208A7004A141F28AA010B192028220849
:10010000A8004A141F288A018207013402340434EB
:1001100008341034203440348034240EC800480C95
:10012000073982078E29A929BD29C829F4291E2A41
:100130000800652A85010730990083160430850080
:10014000FF239000333095000430960099018830E9
:10015000810000308C0083128C010130900020302F
:1001600084008001840A60300406031DB1288830B1
:100170008B00CE015C14581526234A185121CA1B46
:10018000BD285C0E5D06C800480CDF0DDE0DDD0DE0
:10019000DC0D0C1CBD280C10F1308F003819D90B68
:1001A000D2283A21C31CEA2885015808043A031DC5
:1001B000DB284F180514073A031DE028CF188514D3
:1001C000013A031DE5284F1A0516033A031DEA28D4
:1001D000CF1A8516D80BBD2858154B1E0029D40BF5
:1001E00000295C083C39043ED4004F1CFA284F100B
:1001F000051000294F14C31C0514D00B00294B1205
:10020000CB1E1329D50B13295D083C39043ED500BC
:10021000CF1C0D29CF1085101329CF14C31C8514B2
:10022000D10B1329CB124B1F2629D60B26295E088A
:100230003C39043ED6004F1E20294F1205122629B4
:100240004F16C31C0516D20B26294B13CB1F392979
:10025000D70B39295F083C39043ED700CF1E33291C
:10026000CF1285123929CF16C31C8516D30B392915
:10027000CB13BD28D9153308F721330821224318A1
:100280004929051D4629341CEC29D629B41CEC2922
:10029000E129051D4E29341C5B2A282AB41C5B2A3F
:1002A000282A8B134A10230824062506260627062B
:1002B0002806031D9329D9012308A31F7629350693
:1002C000031D932924083606031D9329B81E93297C
:1002D0004A1A93292508A4002608A5002708A60085
:1002E0002808A7008D284A1A9329822903198229F0
:1002F000B81E30060319732937087F394A12031DC7
:100300004A162306031D85298D282308F039703AE3
:100310000319842A230F93298B170800241A9B2979
:10032000240803199629CA138B1708004A13CA1701
:1003300085018B1708002508B7002408123A031915
:10034000B713013A0319B7173708CC000730B423A5
:10035000932924083F3A031D9329A51BB629381871
:10036000B829B71BBA294B18C32993293818B129C2
:10037000B71BB3294B1CCE2993293818CA29B71BA0
:10038000CC294B1CC5294B109329B81CD02193298B
:100390003818BF29B71BC1294B18C5294B149329FD
:1003A0004318262A241EEC294B18E129CB1CDA29F4
:1003B0004B1908003A09CF053908CF04CB144B1567
:1003C0000800CB18E5294B1908003909CF053A0870
:1003D000CF04CB104B1508004B1D08003909CF0581
:1003E0003A09CF054B110800B818D02124080F395D
:1003F000AC04F03A2C05AC00AE002D06AF0043185B
:100400009329C901490883202F05031D102AC90A11
:10041000C91D022A4F08C31C85002C08AD00932972
:100420003B3049078400490883202E0503191B2A05
:100430000008CF04072A0009CF05072A241E252A11
:10044000240EF039AC040F3AFA299329241E5B2AB2
:100450004B190800CF015C080339023ED0005C084C
:100460003C39043ED400DC1B4F144B165D080339A5
:10047000023ED1005D083C39043ED500DD1BCF149F
:10048000CB165E080339023ED2005E083C39043EBA
:10049000D600DE1B4F164B175F080339023ED30010
:1004A0005F083C39043ED700DF1BCF16CB174F083F
:1004B00085004B1508004B1D08008501CF014B122C
:1004C000CB124B13CB134B1108004A1FCB2A4A13F4
:1004D0002608CC00EC302406031DDD2A25084A1E20
:1004E0000319DD2A3423CA18DD2A4A197A2AB423CB
:1004F0002623DD2A023A031DDD2A21302606031DAC
:10050000DD2A75232623DD2ACA1FCD2A4A1FCB2ABE
:10051000CA19EB2A4A132408CC002308F739753A84
:100520000319A62A013A0319A42A023A0319B42A84
:10053000013A0319B82A230803394E073423CA188D
:10054000DD2AA31DC42ABC2A0830A12AA31DAE2A75
:10055000A403A40D240DFC39CE00DD2AA403A40DB0
:10056000240DFC394E06C62A0130A31DC42ADD2AFB
:100570000230A31DC42AD32A4A19D02AB423DF2269
:100580004A134A102623DD2AAE232406031DDD2A42
:10059000DF224A13DD2A4A17DD2ACA134A13DD2A4D
:1005A000023A031DDD2A21302406031DDD2A7523AE
:1005B000DF224A134A102623DD2A8B170800373022
:1005C00085000630C8000030FF3E031DE42AC80B3A
:1005D000E42A850108004A132508CC002318DD2AE7
:1005E00024083423CA18DD2AA319F82A231DDD2A7A
:1005F000231D0C2BA31D042B4A19072BB423DF2228
:100600004A134A102623DD2AAE232506C62A2130A6
:100610002506031DDD2AD72AAE23CC004C308400EA
:10062000073025058320251E1D2BA5198004FF3AC0
:10063000A51D800524083423F42A00050319232B63
:10064000A519C82ADD2AA51DC82ADD2A3030840054
:100650000030CD004D08AE2380004330040603195E
:100660000800840ACD0A2A2BCA104A11003A03193D
:1006700000340C3A03190334013A031904341D3AC7
:1006800003190534013A03190634033A03190734F0
:100690000E3A031908343C3A03190934013A031994
:1006A0000A34033A03190B34013A03190C34073A9C
:1006B00003190D34013A03190E34033A03190F34A8
:1006C000013A031910340F3A03191134013A03198E
:1006D0001234183A031913344A15373A03190134FE
:1006E000013A03190234CA147F340330CC000030BD
:1006F000B423C030CC000530B4230330CC00063026
:10070000B4230430B4230030CC000730B4230630C7
:10071000CC000830B4230130CC000930B4230230BF
:10072000CC000A30B4231030CC000B30B42320307E
:10073000CC000C30B4230030CC000330B4230D3097
:10074000B4230E30B4230F30B4231030B42311304F
:10075000B4231230B4231330B423080083169B0053
:100760001C141A0883120800AE234C060319080053
:100770004C0883169A001C158B1355309D00AA3027
:100780009D009C148B171C119C18C42B831208000D
:02400E00C43FAD
:10420000030014000D0000000300C00003000000C4
:104210000600010002001000200000000000000065
:08422000000000000000000096
:104260006434633463345F34663475346E34633479
:1042700046342E3443346134F1346134643461346F
:10428000333430342F34303434342F343034373402
:00000001FF
